:1000000000308A008D290000FF00030E8301A1004B
:100010007F08A0000A08A8008A01A00E0408A20018
:100020007708A3007808A4007908A5007A08A6003C
:100030007B08A700831383128C308400801C222845
:100040008C183528220884002308F7002408F800BB
:100050002508F9002608FA002708FB0028088A006E
:10006000210E8300FF0E7F0E0900C50ABE0A3E0B5B
:100070003A283D28861606166928BE01BD08031DCC
:1000800044282A08AB0046282908AB00CF014F08B6
:10009000073C031C58282B1C86102B1886140310B1
:1000A000AB0C00000615000006110000CF0A47281F
:1000B000000086150000861186160616BD08031D71
:1000C0006328861264280612BD0A3D08023C031903
:1000D000BD01CF0105184F148518CF1405194F1510
:1000E0008519CF1547084F02031DC5014F08C700EA
:1000F0004508313C031880284F08C4003330C50040
:10010000C80A0319C90A4808E83C031D8E28490893
:10011000033C031D8E28C901C80141148C108A11AB
:1001200022284C30840000080319A5280130F8006B
:10013000F701F70B9928F80B98284A30F700F70BCE
:100140009F2800000000800B9628A9280A30CC00C8
:100150009128013085000F308600831685008601C6
:100160000030F800053883129200FA3083169200AE
:100170000F30F700F71DC628073083128101813048
:1001800084000008C0390F38800083166400813075
:1001900084000008C039770480008C14C0308312BA
:1001A0008B04C529C62983168C14C03083128B0496
:1001B000C729CD014C08093C0318E3284D08CD0A96
:1001C0000A30CC02DA284C08CE002C304E078400CE
:1001D0000008A9002C304D0784000008AA00003454
:1001E00046084A0203190C294608FC3E03180A294E
:1001F000043E0D293230CC00D9200A290A30CC0027
:10020000D9200A290130CC00D9200A29FF30AA00C0
:10021000A9000A294608CA00C8290A148A100A1126
:1002200082070629FA28FE2802294D10430F1929B2
:100230001B294308CC004408F7004C08F8000319B8
:1002400025290310F70CF80B2129771C2929CD103B
:100250002A29CD14430F2D293229CD183129FF30F9
:10026000C3003429CD184D1400304D180130F8006A
:100270000034CC011521F80803194629C301C6082A
:1002800003194429C60146290130C6000130CC00BB
:100290001521F80803194F290130C300C6000230A8
:1002A000CC001521F808031959290230C300033086
:1002B000C6000330CC001521F80803196329033068
:1002C000C3000230C600C92946084B02031984291D
:1002D0004608FC3E03188229043E85290513851330
:1002E000061786138229051785130613861382299C
:1002F000051785170613861782290513851306131C
:10030000861382294608CB00CA290A148A100A11CA
:1003100082077D296E297329782984011F3083057E
:1003200007309F001130AC007730AD004930AE008F
:100330004530AF002730B0008530B1008130B200C9
:100340005730B3000130B4000530B5000330B600BB
:10035000A130B7009930B8006130B9008930BA00D7
:100360008B30BB00FF30BC00BD01BE01BF01C0012E
:10037000C201C300C400C5010130C600C701C801E5
:10038000C901FF30CA00CB00A628D228D328F02804
:10039000392964296400411CD829061CD12906107A
:1003A000D2290614C20A4208643C0319C201411052
:0403B000C6296300F7
:02400E005C3F15
:00000001FF
